:100000000C9463000C948B000C948B000C948B006C
:100010000C948B000C948B000C948B000C948B0034
:100020000C948B000C948B000C948B000C94E110BE
:100030000C948B000C948B000C948B000C948B0014
:100040000C94FC270C948B000C94502A0C948B007D
:100050000C948B000C948B000C948B000C948B00F4
:100060000C948B000C948B000000000024002700EF
:100070002A0000000000250028002B0000000000DE
:1000800023002600290004040404040404040202DA
:100090000202020203030303030301020408102007
:1000A0004080010204081020010204081020000012
:1000B0000007000201000003040600000000000029
:1000C00000000706E12B11241FBECFEFD8E0DEBFF2
:1000D000CDBF11E0A0E0B1E0E4ECFDE502C0059089
:1000E0000D92AE39B107D9F713E0AEE9B1E001C026
:1000F0001D92A037B107E1F710E0C6ECD0E004C0D4
:100100002297FE010E94A52EC23CD107C9F70E948A
:100110001B2C0C94E02E0C940000CF93DF93BC01B9
:100120008230910510F462E070E0A0916E03B0910E
:100130006F03ED01E0E0F0E040E050E021C0888195
:1001400099818617970769F48A819B81309719F006
:100150009383828304C090936F0380936E03FE01A8
:1001600034C06817790738F44115510519F0841720
:10017000950708F4AC01FE018A819B819C01E9018D
:100180002097E9F641155105A9F1CA01861B970B85
:10019000049708F4BA01E0E0F0E02AC08D919C9148
:1001A000119784179507F9F46417750781F412966F
:1001B0008D919C911397309719F09383828304C09B
:1001C00090936F0380936E03FD0132964CC0CA0179
:1001D000861B970BFD01E80FF91F6193719302973E
:1001E0008D939C9340C0FD01828193819C01D90134
:1001F0001097A1F680916C0390916D03892B41F4C7
:10020000809166019091670190936D0380936C03D8
:1002100040916801509169014115510541F44DB774
:100220005EB78091640190916501481B590B209144
:100230006C0330916D03CA01821B930B86179707DD
:1002400080F0AB014E5F5F4F8417950750F0420F6F
:10025000531F50936D0340936C03F90161937193A5
:1002600002C0E0E0F0E0CF01DF91CF910895CF939D
:10027000DF93009709F450C0EC0122971B821A8289
:10028000A0916E03B0916F03109709F140E050E028
:10029000AC17BD0708F1BB83AA83FE012191319100
:1002A000E20FF31FAE17BF0779F48D919C91119760
:1002B000280F391F2E5F3F4F3983288312968D9167
:1002C0009C9113979B838A834115510571F4D093B8
:1002D0006F03C0936E0320C012968D919C9113976B
:1002E000AD01009711F0DC01D3CFFA01D383C283B3
:1002F00021913191E20FF31FCE17DF0769F4888156
:100300009981280F391F2E5F3F4FFA0131832083D7
:100310008A819B8193838283DF91CF910895A0E0AE
:10032000B0E0E5E9F1E00C94B12EEC01A880B980D1
:10033000CA80DB80A114B104C104D10441F484E279
:10034000A82E89EDB82E8BE5C82E87E0D82EC601E1
:10035000B5012DE133EF41E050E00E94742E27EA11
:1003600031E440E050E00E94142E7B018C01C60174
:10037000B5012DE133EF41E050E00E94742ECA0137
:10038000B9012CEE34EF4FEF5FEF0E94142E6E0D8B
:100390007F1D801F911F97FF04C0615070408040F7
:1003A0009048688379838A839B839B01AC015F7744
:1003B000B901CA01CDB7DEB7EAE00C94CD2E0E9498
:1003C0008F0108958AE691E00E948F01089560935D
:1003D0006A0170936B0180936C0190936D01089595
:1003E000FB01DC0104C08D910190801921F4415082
:1003F0005040C8F7881B990B0895FB01DC01019060
:100400000D920020E1F70895F999FECF72BD61BD0C
:10041000F89A80B50895F999FECF1FBA72BD61BDF3
:1004200040BD0FB6F894FA9AF99A0FBE0895FC01F0
:1004300083E791E0918380838FEF8283148213821C
:10044000168215820895DF93CF930F92CDB7DEB752
:10045000FC016983A081B18114962D913C9115977F
:10046000BE016F5F7F4F41E050E0F90109950F90A9
:10047000CF91DF9108950F931F93CF93DF938C015A
:10048000FC0182818F3F89F0982F80E08F5F9B4F26
:100490000E940B0CF8018281D82FC0E0CE018F5F43
:1004A0009B4F0E942A0C8823A9F7DF91CF911F91BF
:1004B0000F9108950F931F93CF93DF93EC018A81DF
:1004C0008F3F79F0CE0160E10E943B028A81182FB4
:1004D00000E0C8018E5F9B4F6FEF0E940B0C8FEF07
:1004E0008A83DF91CF911F910F910895FC01828142
:1004F0008F3F11F480E008950E945F0E08950E94DE
:10050000760290E0882309F491E0892F0895FF9204
:100510000F931F93CF93DF93EC010E947F028823F8
:10052000C1F48A81982F80E08C5D9B4F0E942A0C39
:10053000F82E8B831C828A81182F00E0C8018B5D06
:100540009B4F0E942A0C3F2D20E0280F311D3C8339
:100550002B83DF91CF911F910F91FF900895CF9240
:10056000DF92EF92FF920F931F93CF93DF93EC01F3
:100570007B016A010E947F028823C1F58A81982F3E
:1005800080E0845F9B4FF70160810E940B0C8A81A1
:10059000182F00E0C801835F9B4FF70161810E9423
:1005A0000B0C8A81182FC801825F9B4FF701628173
:1005B0000E940B0C8A81182FC801815F9B4FF701A5
:1005C00063810E940B0C8A81182FC801805F9B4FAA
:1005D0006D2D0E940B0C8A81182FC8018F5E9B4FD6
:1005E0006C2D0E940B0CCE010E948702DF91CF91EF
:1005F0001F910F91FF90EF90DF90CF900895CF92D1
:10060000DF92EF92FF920F931F93CF93DF93EC0152
:100610007B016A010E947F028823C9F58A81982F95
:1006200080E0845F9B4FF70160810E940B0C8A8100
:10063000182F00E0C801835F9B4FF70161810E9482
:100640000B0C8A81182FC801825F9B4FF7016281D2
:100650000E940B0C8A81182FC801815F9B4FF70104
:1006600063810E940B0C8A81182FC801805F9B4F09
:100670006D2D0E940B0C8A81182FC8018F5E9B4F35
:100680006C2D0E940B0CCE0164E00E943B02DF91B6
:10069000CF911F910F91FF90EF90DF90CF90089531
:1006A000CF93DF93EC010E947F028823F1F48A81CB
:1006B000982F80E08E5F9B4F0E942A0C9A8184FDC8
:1006C0000EC080E08E5F9B4F0E942A0C83FF0DC0FE
:1006D0008A81982F80E08E5F9B4F68E104C080E0A4
:1006E0008E5F9B4F60E10E940B0C81E0DF91CF9108
:1006F00008950F931F93CF93DF93EC010E947F0225
:100700008823A9F48A81982F80E06C818C5D9B4FAF
:100710000E940B0C8A81182F00E0C8018B5D9B4F53
:100720006B810E940B0CCE0160E20E943B02DF91C4
:10073000CF911F910F910895DF92EF92FF920F9347
:100740001F93CF93DF93EC01D62E7A01122F1A82DA
:1007500008C0CE010E947F02882331F48A818F5F16
:100760008A838A818430A8F30A81043019F48FEFD8
:100770008A830DC0E114F10431F4E02EFF2480E0FF
:1007800094E0E80EF91E8D2D8150853010F080E048
:1007900021C0CE010E945A020A831D2980E0902FB9
:1007A0009C5F612F0E940B0C8A81182F00E0C8010A
:1007B0008C5F9B4F6F2D0E940B0C8A81182FC801F4
:1007C0008B5F9B4F6E2D0E940B0CCE0161E00E944F
:1007D0003B0281E0DF91CF911F910F91FF90EF904D
:1007E000DF900895AB0162E020E00E949C03089531
:1007F000AB0161E020E00E949C030895CF93DF935A
:10080000EC010E947F02882319F020E030E004C050
:100810008A810E94A90E9C01C901DF91CF910895A0
:10082000AF92BF92CF92DF92FF920F931F93CF931D
:10083000DF93EC015B016A014115510509F440C0E9
:100840000E947F028823E1F58A81982F80E0885DED
:100850009B4F0E942A0CF82E8D831E828A81182FAE
:1008600000E0C801875D9B4F0E942A0C3F2D20E0CD
:10087000B901680F711D7E836D83A114B10429F045
:100880008A81A50196010E94370F2D813E812C0D92
:100890003D1D3E832D838A81982F80E0885D9B4F8C
:1008A000632F0E940B0C8A81182F00E0C801875D1E
:1008B0009B4F6D810E940B0CCE0160E40E943B02B5
:1008C000DF91CF911F910F91FF90DF90CF90BF905C
:1008D000AF900895CF92DF92EF92FF920F931F9304
:1008E000DF93CF93CDB7DEB728970FB6F894DEBF6E
:1008F0000FBECDBF8C017B016A010E947F0288235D
:1009000019F020E030E025C0C8010E94FE030897DE
:10091000D8F3C801BE016F5F7F4F48E050E00E94EE
:1009200010048981F70180838A8181838B8182838E
:100930008C8183839D8180E02E81820F911DF60141
:10094000918380839F8180E02885AC01420F511DF7
:100950009A01C90128960FB6F894DEBF0FBECDBF2D
:10096000CF91DF911F910F91FF90EF90DF90CF908B
:100970000895AB0160E070E00E9410040895CF93E9
:10098000DF93DB010D900020E9F71197A61BB70B51
:10099000EC01E881F9810480F581E02DAD01099534
:1009A000DF91CF910895CF92DF92EF92FF920F9354
:1009B0001F93CF93DF93EC016B018A010E947F02AA
:1009C000882339F58A810E94020C8017910720F450
:1009D0008A810E94020C8C018A810E94670E7C0130
:1009E000CE010E947602873121F08C3111F08232E3
:1009F00081F4E016F10680F34B815C818A81B601B7
:100A000098010E94EF0E8B819C81800F911F9C8327
:100A10008B83DF91CF911F910F91FF90EF90DF902B
:100A2000CF900895DF93CF930F92CDB7DEB7FC013F
:100A30006983A081B18114962D913C911597BE01D7
:100A40006F5F7F4F41E050E0F90109950F90CF9122
:100A5000DF91089508960E94FE030895CF93DF93D7
:100A6000EC012896CE010E947602843171F0882331
:100A700061F0883151F08C3131F4CE010E94FE03D7
:100A800020E0892B19F021E001C020E0822FDF91C6
:100A9000CF9108950F931F938C01085F1F4FC801DA
:100AA0000E94FE03BC01C8010E94B9041F910F916E
:100AB00008950F931F93DF93CF930F92CDB7DEB7B7
:100AC0008C01085F1F4FC8010E94FE03892B19F497
:100AD0002FEF3FEF0BC0C801BE016F5F7F4F41E0BA
:100AE00050E00E9410048981282F30E0C9010F9046
:100AF000CF91DF911F910F910895CF92DF92EF92E6
:100B0000FF920F931F938B016A0128E0E22EF12CD4
:100B1000E80EF91EC7010E948702C701B801A601AD
:100B20000E94D304C7010E9479031F910F91FF9087
:100B3000EF90DF90CF900895CF93DF93DB010D907E
:100B40000020E9F71197A61BB70BEC01E881F981AA
:100B50000480F581E02DAD010995DF91CF910895D5
:100B60000F931F93CF93DF93EC018C01085F1F4F0E
:100B70006A817B81C8010E94F8038823F1F06C81AF
:100B80007D814E815F81C8010E94FF0210C061E03B
:100B900070E080E090E00E947828C8010E94760210
:100BA000882329F4C8010E945A0280E006C0C801C7
:100BB0000E947602873159F781E0DF91CF911F9132
:100BC0000F910895AF92BF92CF92DF92EF92FF9272
:100BD0000F931F938C017B016A0159018DE791E00E
:100BE000F80191838083C80108960E941702F801DA
:100BF000F582E482D782C682B382A2821F910F91CE
:100C0000FF90EF90DF90CF90BF90AF9008958DEB65
:100C100091E00E9417020895CF93DF93FB01EC014E
:100C20008A8D9B8DAC8DBD8D80839183A283B38390
:100C3000DF91CF910895CF93DF93FB01EC018E8973
:100C40009F89A88DB98D80839183A283B383DF911F
:100C5000CF910895CF93DF93FB01EC018A899B89A3
:100C6000AC89BD8980839183A283B383DF91CF91C7
:100C70000895CF93DF93FB01EC018E859F85A889B2
:100C8000B98980839183A283B383DF91CF91089543
:100C9000CF93DF93FB01EC018A859B85AC85BD85F5
:100CA00080839183A283B383DF91CF9108952F92A4
:100CB0003F924F925F926F927F928F929F92AF92EC
:100CC000BF92CF92DF92EF92FF920F931F93DF9329
:100CD000CF93CDB7DEB727970FB6F894DEBF0FBE20
:100CE000CDBF5C013A014B011B821A820E9444284D
:100CF0007B018C012EE1422E512C4A0C5B1C0EC054
:100D00000E9444286E197F09800B910B66167706A6
:100D10008806990618F4FF24FA94B9C0C2010E940B
:100D2000FE03089768F3C201BE016C5F7F4FAE01FE
:100D30004E5F5F4F0E946A043C0182E290E00E9495
:100D40008D00982E892EC82ED92EC201692D782D9E
:100D500042E250E00E941004D6018C91823009F0EA
:100D600083C08A819B818334910509F07DC0B501E0
:100D70006C5F7F4FC6014C9646E050E00E94F00148
:100D8000009709F083C0F601E480F58006811781A1
:100D9000D5016D917D918D919C910E94C70BE616B6
:100DA000F7060807190709F071C08BC0FD013196DD
:100DB0008C91863051F1873048F4813099F0813040
:100DC00008F447C0833009F043C013C0853339F0BD
:100DD0008633F0F1863311F18F3FD1F53AC061913E
:100DE000F08037C061912081318142815381D801E7
:100DF00006C061912081318142815381D3012D93BD
:100E00003D934D935C93139724C011966C9131964A
:100E10002081318142815381D401F1CF6191D5018B
:100E20002D913D914D915C91211531054105510563
:100E300049F08C819D81AE81BF81281739074A070F
:100E40005B0739F42081318142815381D501D7CFAD
:100E50006191DF01A60FB11DA215B30508F4A6CF5D
:100E6000C6010E94370109C0FF2407C0C201B801B2
:100E700041E050E00E94100403C08E010F5F1F4F3D
:100E8000C2010E94FE03892B89F701C0FF248F2D28
:100E900027960FB6F894DEBF0FBECDBFCF91DF917E
:100EA0001F910F91FF90EF90DF90CF90BF90AF9088
:100EB0009F908F907F906F905F904F903F902F907A
:100EC0000895F60180899189A289B389F501828705
:100ED0009387A487B587C2016EEC70E00E94B904C5
:100EE000892D982D0E9437018301005F1040C801B1
:100EF0000E948D006C01C201B601A8010E9410047D
:100F00001601200E311E8501025F1F4F92E1692EEE
:100F1000712C6A0C7B1C8AE1882E912C8A0C9B1CFC
:100F200086E190E0A80EB91ED601FF2460E094CFC0
:100F30002F923F924F925F926F927F928F929F92E9
:100F4000AF92BF92CF92DF92EF92FF920F931F93D7
:100F5000DF93CF93CDB7DEB767970FB6F894DEBFB8
:100F60000FBECDBF6C016F8B8A018FEF8B838C839B
:100F70008D838E835EE1A52EB12CAC0CBD1CC5010A
:100F8000BE016D5F7F4F43E450E00E94AF0280E2FC
:100F900090E00E948D007C0180E2F70111928A9519
:100FA000E9F781E0F70181933F01F7018183970120
:100FB0002E5F3F4F3E8B2D8B86E08283C7010396C9
:100FC0009C8B8B8B1382F601619171918191919130
:100FD0004F010E94C70B6F83788789879A8744E007
:100FE000442E512C4E0C5F1CF7016483758386835D
:100FF000978338E0232E312C2E0C3F1C108797014D
:10100000275F3F4F3A8B298B018780E090E80E9451
:10101000CA0B9A838983F7013A96F88BEF87F70119
:1010200093878287C501B7014CE150E00E94D30449
:10103000D701F40186E001900D928150E1F7C501DE
:10104000B70140E150E00E94D30480E2F701119221
:101050008A95E9F700E010E0C501B70140E250E0F1
:101060000E94D3040F5F1F4F06301105A9F793E6C6
:10107000F701908382E8F301808383E5ED89FE899F
:101080008083EB89FC89908385E3F201808397015B
:101090002B5F3F4F3E872D8791E0F70195839701A6
:1010A0002A5F3F4F3C872B873F8936838701095F43
:1010B0001F4F8DE3878387E0F1018083E989FA89F7
:1010C0009083AF85B889F40186E001900D9281503C
:1010D000E1F78CE0F701808B89E0818BC7014296B4
:1010E00060E071E00E94FD01F6018781F701808FC9
:1010F000F6018085F701818FF6018185F701828FE6
:10110000C501B7014BE150E00E94D304FF89F330E1
:10111000B9F582E3F701808394E0F3019083F6014F
:101120008285ED89FE898083F6018385EB89FC89C0
:101130008083F6018485F2018083F6018585ED8543
:10114000FE85808386E3EB85FC858083F8019083B0
:10115000F6018689F1018083F6018789E989FA8998
:101160008083F601808DEF85F8898083F601818D7B
:10117000F7018387C501B7014CE050E00E94D3041A
:1011800087E3F701808396E0F301908381E0ED89A6
:10119000FE89808383E0EB89FC898083F201908360
:1011A0008FE0ED85FE8580838AE3EB85FC85808377
:1011B0008BE3F80180838FEFF1018083C501B701D4
:1011C00049E050E00E94D304E114F10419F0C70192
:1011D0000E943701C5010E947903C5010E94500396
:1011E0008823D9F367960FB6F894DEBF0FBECDBF44
:1011F000CF91DF911F910F91FF90EF90DF90CF90F3
:10120000BF90AF909F908F907F906F905F904F9026
:101210003F902F9008952F923F924F925F926F923E
:101220007F928F929F92AF92BF92CF92DF92EF9276
:10123000FF920F931F93DF93CF9300D000D000D085
:10124000CDB7DEB76C0129833A834B835C832701DA
:101250003801E4E0AE2EB12CA80EB91E8AE1F501EA
:1012600011928A95E9F7D501FB0186E001900D9274
:101270008150E1F70E94D70DC5010E94170E7AE058
:10128000272E312C2C0C3D1CC1010E94410E85E5FE
:1012900065E50E94A20C6EE1E62EF12CEC0CFD1C23
:1012A000C70164E470E00E94F203882319F42FEF71
:1012B0003FEF80C00E9444284B015C0110E01E8279
:1012C0001D821123F9F4F60180819181A281B381FD
:1012D0000196A11DB11D80839183A283B3830E94D7
:1012E0004428681979098A099B0928EE33E040E00F
:1012F00050E00E94522EC60161E0A9010E949807A9
:1013000011E02BC01130D1F4C601B301A2010E943B
:1013100057068230F9F40E944428681979098A092D
:101320009B0928EE33E040E050E00E94522EC601B7
:1013300063E0A9010E94980712E00FC0123069F41F
:10134000C601B301A2010E945706853009F45FC0AF
:10135000863011F08F3F09F410E02D813E8121305D
:10136000310509F450C00E944428681979098A0996
:101370009B0929813A814B815C81261737074807F1
:10138000590708F040C0F60180819181A281B381A4
:101390000196A11DB11D80839183A283B383C701F0
:1013A0000E945A022D813E812130310531F08D811C
:1013B0009E819C013E832D830BC0C1010E94410E82
:1013C000C60142960E94DB0DC6010E960E94F90DE1
:1013D0008D819E8126960FB6F894DEBF0FBECDBFDD
:1013E000CF91DF911F910F91FF90EF90DF90CF9001
:1013F000BF90AF909F908F907F906F905F904F9035
:101400003F902F900895133009F05BCFBCCF13E0CD
:1014100041E050E05E834D83A0CFEF92FF920F93A7
:101420001F93DF93CF930F92CDB7DEB78C010C5F84
:101430001F4F7E010894E11CF11CC801B70141E077
:1014400050E00E9410046981662379F0862F807C29
:10145000803C31F4C80161E070E00E94B90405C02D
:10146000C80170E00E94B904E8CF0F90CF91DF91DE
:101470001F910F91FF90EF900895CF93DF93FB01A1
:10148000EC018B899C89AD89BE8980839183A2837D
:10149000B383DF91CF9108959C01FA01DC0152964C
:1014A0007C936E93519780819181A281B381F901E0
:1014B00080839183A283B3830895AF92BF92DF921A
:1014C000EF92FF920F931F93DF93CF93CDB7DEB7C9
:1014D0002C970FB6F894DEBF0FBECDBF8C0184E011
:1014E000E82EF12CE00EF11EC7010E94FE03449786
:1014F00008F45FC0B801655F7F4FA801415F5F4F8F
:10150000C7010E946A04C7015E010894A11CB11CB6
:10151000B5014CE050E00E941004DC802FE0D222A4
:1015200099F089E593E067E071E00E94592C89E524
:1015300093E06C8140E150E00E94692DC7010E9458
:101540005A028D2D805F4BC0D884C8010E940D0ABD
:10155000C70164E070E00E94B90424C0C8010E9481
:101560000D0AC701B5014AE050E00E9410048A81CB
:10157000813091F48D819E81F801908F878B0D5E73
:101580001F4FC701B80144E050E00E941004C7019A
:101590000E945A0281E023C06A85C70170E00E9460
:1015A000B904DA941D14D4F2C7010E945A0282E0F1
:1015B00016C00E944428F801238D348D458D568D28
:1015C000621B730B840B950B6958734180409040EC
:1015D00010F480E004C0C7010E945A0283E02C96F8
:1015E0000FB6F894DEBF0FBECDBFCF91DF911F9134
:1015F0000F91FF90EF90DF90BF90AF900895AF9262
:10160000BF92CF92DF92FF920F931F93DF93CF93FE
:10161000CDB7DEB762970FB6F894DEBF0FBECDBF71
:101620006C01DE011796E8E8F1E08CE001900D9284
:101630008150E1F7DE011296E3E8F1E085E00190E8
:101640000D928150E1F7198286010C5F1F4FC8018E
:1016500060E070E00E94F203882309F45EC0C801D4
:10166000B60145E350E00E94AF02C801BE01695FC8
:101670007F4F4CE050E00E94D304FF24F3945E01BE
:101680000894A11CB11C22C089818F5F8983240F1B
:10169000351FF901A081AE3211F0AA23B1F4C801BF
:1016A000B50141E050E00E94D30449818F2D90E0C4
:1016B000841B9109F60161897289680F791FC8013D
:1016C00050E00E94D3041982F394F3944F2D50E01C
:1016D000F60121893289F90101900020E9F731975B
:1016E000E21BF30BE417F50778F6C801BE016E5F45
:1016F0007F4F45E050E00E94D304C8010E94790367
:10170000C8010E9450038823D9F30E944428F6019F
:10171000638F748F858F968F81E062960FB6F894F1
:10172000DEBF0FBECDBFCF91DF911F910F91FF9014
:10173000DF90CF90BF90AF90089504960E9417025B
:101740000895AF92BF92CF92DF92EF92FF920F93E4
:101750001F937B016A0159010E94D70D85E565E55C
:101760000E94A20CC7010E94170EC6010E94410EE2
:10177000C5010E94DB0DC8010E94F90D1F910F9158
:10178000FF90EF90DF90CF90BF90AF9008950E94B0
:10179000D50B08950E94CD0B0895582F40E0292FB6
:1017A00030E0242B352BC9010895EF92FF920F935F
:1017B0001F93562F442733272227E92EFF24002783
:1017C0001127E22AF32A042B152B272F30E040E0C3
:1017D00050E0A90133272227E22AF32A042B152BF4
:1017E000672F782F892F9927607080709070E62A74
:1017F000F72A082B192BB701C8011F910F91FF90F1
:10180000EF900895E82FF0E0EE0FFF1FEB52FE4F30
:10181000808191810895282F84B18C6284B92A9A9D
:1018200085B1877D85B980E58CBD2A9880EF8EBD16
:101830000DB407FEFDCF9EBD0DB407FEFDCF2EBD3E
:101840000DB407FEFDCF6EBD0DB407FEFDCF2A9A85
:1018500081E00895282F84B18C6284B92A9A85B1D9
:10186000877D85B980E58CBD2A988FE08EBD0DB44B
:1018700007FEFDCF9EBD0DB407FEFDCF2EBD0DB4FE
:1018800007FEFDCF1EBC0DB407FEFDCF8EB52A9A14
:101890000895DC0184B18C6284B92A9A85B1877D70
:1018A00085B980E58CBD20E030E090EF19C02A9822
:1018B0009EBD0DB407FEFDCFBEBD0DB407FEFDCF2E
:1018C000AEBD0DB407FEFDCFFB01E20FF31F80811B
:1018D0008EBD0DB407FEFDCF2A9A2F5F3F4F1196A4
:1018E0002417350720F3CA010895DC0184B18C6206
:1018F00084B92A9A85B1877D85B980E58CBD20E0C1
:1019000030E09FE01AC02A989EBD0DB407FEFDCFBF
:10191000BEBD0DB407FEFDCFAEBD0DB407FEFDCFBD
:101920001EBC0DB407FEFDCF8EB5FB01E20FF31F09
:1019300080832A9A2F5F3F4F11962417350718F39B
:10194000CA0108952F923F924F925F926F927F92B9
:101950008F929F92AF92BF92CF92DF92EF92FF92BF
:101960000F931F93DF93CF9300D000D0CDB7DEB796
:10197000182F062F8BE190E0612F0E940B0C8AE15B
:1019800090E0602F0E940B0C80E090E49093E601C1
:101990008093E50180E090E69093EE018093ED0165
:1019A00065ED71E08DED91E09C838B83FDECCF2E96
:1019B000F1E0DF2EE5ECEE2EE1E0FE2E662477244A
:1019C000AA24BB248824992440E050E0E12FF0E0D1
:1019D000FA83E983202E3324FB0111821082EB81EC
:1019E000FC8111821082F0E08F16F0E29F06DCF598
:1019F00089819A81042E02C0959587950A94E2F711
:101A00008370907081309105A1F0823091051CF4B3
:101A1000892B39F028C08230910599F0039719F588
:101A200018C080E094E0FB01918380838FEF93E006
:101A300017C080E098E0FB01918380838FEF97E0EF
:101A40000FC080E090E1FB01918380838FEF9FE0E6
:101A500007C080E090E2FB01918380838FEF9FE1DC
:101A6000F7019183808390E0691690E279060CF08B
:101A70003EC0C101042E02C0959587950A94E2F7F5
:101A80008370907081309105A9F0823091051CF42B
:101A9000892B39F02CC082309105A9F0039739F5D4
:101AA0001BC080E094E0EB81FC81918380838FEF09
:101AB00093E01AC080E098E0EB81FC819183808301
:101AC0008FEF97E011C080E090E1EB81FC81918382
:101AD00080838FEF9FE008C080E090E2EB81FC8183
:101AE000918380838FEF9FE1F60191838083FB01D7
:101AF00040805180EB81FC8100811181A114B104EF
:101B0000F1F0FA01EB51FE4FDA01AD52BE4F8D916B
:101B10009C91329122913296820F931F9183808300
:101B2000FA01E351FE4FDA01A552BE4F8D919C910F
:101B3000329122913296820F931F91838083089471
:101B4000A11CB11C6E5F7F4F4E5F5F4F8B819C81EC
:101B500002969C838B83E2E0F0E0CE0EDF1EEE0E59
:101B6000FF1EF4E0AF16B10429F0840C951C600E42
:101B7000711E32CF0F900F900F900F90CF91DF9189
:101B80001F910F91FF90EF90DF90CF90BF90AF909B
:101B90009F908F907F906F905F904F903F902F908D
:101BA0000895682F80E090E80E940B0C089580E86B
:101BB0000E94D10D08950F931F938C0181E090E056
:101BC000F80160810E940B0C82E090E0F8016181D5
:101BD0000E940B0C83E090E0F80162810E940B0CE4
:101BE00084E090E0F80163810E940B0C1F910F913B
:101BF00008950F931F938C0185E090E0F8016081B8
:101C00000E940B0C86E090E0F80161810E940B0CB1
:101C100087E090E0F80162810E940B0C88E090E080
:101C2000F80163810E940B0C1F910F9108950F938F
:101C30001F938C0189E090E0F80160810E940B0CF9
:101C40008AE090E0F80161810E940B0C8BE090E04B
:101C5000F80162810E940B0C8CE090E0F801638136
:101C60000E940B0C8DE090E0F80164810E940B0C47
:101C70008EE090E0F80165810E940B0C1F910F919E
:101C800008950F931F938C018FE090E0F80160811D
:101C90000E940B0C80E190E0F80161810E940B0C26
:101CA00081E190E0F80162810E940B0C82E190E0FA
:101CB000F80163810E940B0C1F910F91089590E031
:101CC000982F88278D5F9B4F0E942A0C08958F9232
:101CD0009F92AF92BF92CF92DF92EF92FF920F93BB
:101CE0001F93CF93DF9390E0982F8827805E9B4FC0
:101CF0004C015C010894A11CB11CC0E0D0E0C401FF
:101D00000E942A0CF82EEE24C5010E942A0C6701BD
:101D1000C80ED11CC114D10459F0C4010E942A0C70
:101D2000182F00E0C5010E942A0CE801C80FD11D40
:101D3000CC15DD0521F7CE01DF91CF911F910F91D9
:101D4000FF90EF90DF90CF90BF90AF909F908F90DB
:101D500008958F929F92AF92BF92CF92DF92EF92AF
:101D6000FF920F931F93CF93DF9390E00496982FE9
:101D7000882716E2812E912C880E991EB7E2AB2E91
:101D8000B12CA80EB91EC0E0D0E0C4010E942A0CFC
:101D9000F82EEE24C5010E942A0C6701C80ED11C42
:101DA000C114D10459F0C4010E942A0C182F00E07C
:101DB000C5010E942A0CE801C80FD11DCC15DD0514
:101DC00021F7CE01DF91CF911F910F91FF90EF90FE
:101DD000DF90CF90BF90AF909F908F900895CF925B
:101DE000DF92EF92FF920F931F93CF93DF937B01CC
:101DF000E901E82FF0E0EE0FFF1FDF01AB53BE4F0C
:101E00008D919C914823592385EEC82E81E0D82ED0
:101E1000CE0EDF1ED6012D913C91240F351FEB52C3
:101E2000FE4F0190F081E02DCA018C0F9D1FE81735
:101E3000F90780F48F01041B150BC901A8010E944A
:101E4000490CC01BD10BF601808191810E0D1F1D25
:101E5000B80101C0C901AE010E94490CDF91CF91C8
:101E60001F910F91FF90EF90DF90CF900895CF9248
:101E7000DF92EF92FF920F931F93CF93DF937A013C
:101E8000E901E82FF0E0EE0FFF1FDF01A353BE4F83
:101E90008D919C91682379234DEEC42E41E0D42E80
:101EA000CE0EDF1ED6012D913C91260F371FE35237
:101EB000FE4F0190F081E02DCE01860F971FE817AD
:101EC000F90788F48F01061B170BC901B701A80198
:101ED0000E94750CC01BD10BF601808191810E0D03
:101EE0001F1DB80102C0C901B701AE010E94750CE7
:101EF000DF91CF911F910F91FF90EF90DF90CF90E6
:101F00000895DF93CF9300D0CDB7DEB720916C0357
:101F100030916D03CE0101962115310519F48057DA
:101F2000934002C0821B930B9A83898389819A8193
:101F30000F900F90CF91DF910895FC018091F501F2
:101F40008C3090F480838F5F8093F501815090E016
:101F5000FC01EE0FFF1FE80FF91FEA50FE4F88EB60
:101F60009BE09283818308958FEF80830895FC0125
:101F700020812C30B8F58181992787FD909548E81C
:101F800050E0481B590B440F551F440F551F641751
:101F9000750784F08281992787FD909548E552E086
:101FA000481B590B440F551F440F551F64177507E5
:101FB0000CF4AB0142505040CA01AA2797FDA095EE
:101FC000BA2F880F991FAA1FBB1F4FB7F89430E094
:101FD000F901EE0FFF1FE20FF31FEA50FE4F92834D
:101FE00081834FBF0895AF92BF92CF92DF92EF925D
:101FF000FF920F931F93CF93DF93EC019B0182E03D
:10200000603278070CF048C077FF03C020E030E072
:1020100005C0653B710514F024EB30E000D000D022
:10202000B901882777FD8095982F2981332727FDCF
:102030003095E8E8AE2EB12CA21AB30AAA0CBB1C4C
:10204000AA0CBB1CCC24B7FCC094DC2CEA81FF2773
:10205000E7FDF09528E532E02E1B3F0B220F331FE2
:10206000220F331F442737FD4095542FEDB7FEB79D
:10207000218332834383548320E030E040E050E00A
:1020800004EBE02EF12C012D112D0E94832D9B01DC
:102090000F900F900F900F90CE01B9010E94B70FD3
:1020A000DF91CF911F910F91FF90EF90DF90CF9034
:1020B000BF90AF900895CF92DF92EF92FF921F935F
:1020C000CF93DF93EC01162F7A01690188818C3060
:1020D00008F064C0862F61E00E945329888190E057
:1020E000FC01EE0FFF1FE80FF91FEA50FE4F1F73B0
:1020F0008081807C812B808380E292E08E199F0911
:1021000064E070E00E943F2E698380E699E08C19BC
:102110009D0964E070E00E943F2E6A83A8818A2FA7
:102120006CE00E94332E682F70E0AB01440F551F06
:10213000460F571F440F551F440F551F20E030E036
:10214000C901840F951FFC01EE0FFF1FE80FF91F57
:10215000EA50FE4F808186FD15C02F5F3F4F2C3027
:10216000310571F724C01092800082E080938100D5
:102170001092850010928400B19A80916F00826065
:1021800080936F008A2F90E0FC01EE0FFF1FE80F95
:10219000F91FEA50FE4F8081806480838881DF913F
:1021A000CF911F91FF90EF90DF90CF900895672B14
:1021B000D1F2E8CF40E252E020E639E00E945B1025
:1021C00008951F920F920FB60F9211242F933F93F1
:1021D0004F935F936F937F938F939F93AF93BF932F
:1021E000EF93FF9380911A0287FF05C0109285003C
:1021F000109284002BC020911A02332727FD3095BE
:102200008091F50190E02817390704F580911A02B2
:10221000992787FD9095FC01EE0FFF1FE80FF91F2E
:10222000EA50FE4F808186FF11C080911A029927E3
:1022300087FD9095FC01EE0FFF1FE80FF91FEA5094
:10224000FE4F80818F7360E00E94732980911A0293
:102250008F5F80931A0220911A02332727FD309551
:102260008091F50190E0281739070CF04EC080915D
:102270001A028C300CF049C0209184003091850006
:1022800080911A02992787FD9095FC01EE0FFF1FA0
:10229000E80FF91FEA50FE4F81819281280F391F04
:1022A000309389002093880080911A02992787FD36
:1022B0009095FC01EE0FFF1FE80FF91FEA50FE4F4B
:1022C000808186FF2AC080911A02992787FD909508
:1022D000FC01EE0FFF1FE80FF91FEA50FE4F80814F
:1022E0008F7361E00E94732918C080E49CE905C0E7
:1022F000809184009091850004969093890080934A
:1023000088008FEF80931A0208C08091840090911A
:10231000850084549C4948F3EBCFFF91EF91BF9126
:10232000AF919F918F917F916F915F914F913F916D
:102330002F910F900FBE0F901F90189508958091C8
:10234000B302882319F061E00E9473290895BF92B7
:10235000CF92DF92EF92FF920F931F93CF93DF9371
:102360006C01B62E79018A018091B402882349F567
:1023700053C08091B40261E00E9473296091BA0257
:102380007091BB0280E090E00E9478288091B402B6
:1023900060E00E9473296091BC027091BD0280E0F0
:1023A00090E00E9478282196CC15DD0510F360910D
:1023B000BE027091BF0280E090E00E947828BB20AE
:1023C00019F0C0E0D0E0F0CF1E141F041006110673
:1023D0001CF58091BC029091BD022091BA0230910F
:1023E000BB02820F931F9C01C29EC001C39E900D31
:1023F000D29E900D1124A0E0B0E0E81AF90A0A0B71
:102400001B0B8091BE029091BF02A0E0B0E0E81AE1
:10241000F90A0A0B1B0BD5CFDF91CF911F910F91BA
:10242000FF90EF90DF90CF90BF900895EF92FF92D2
:102430000F931F93CF93DF93EC017A018B0127C099
:102440006AE070E080E090E00E94782886EF9FEFDD
:10245000AFEFBFEFE80EF91E0A1F1B1F1E141F046B
:1024600010061106A4F089E090E060E020E030E082
:1024700040E050E00E94A7110E949F1189E090E087
:1024800061E020E030E040E050E00E94A711CE0182
:102490000E942A05892BA1F2DF91CF911F910F9104
:1024A000FF90EF9008952F923F924F925F926F921C
:1024B0007F928F929F92AF92BF92CF92DF92EF92D4
:1024C000FF920F931F93DF93CF93CDB7DEB7C4581E
:1024D000D2400FB6F894DEBF0FBECDBF8CE192E0C4
:1024E00066E171E00E94FD018EE991E060E070E03C
:1024F0000E940402803811F00C9475278EE991E057
:1025000061E270E00E940402803811F00C9475279B
:102510008EE991E064E870E00E940402803811F0D6
:102520000C9475278EE991E069E870E00E9404023E
:10253000803811F00C9475278EE991E06CE870E01A
:102540000E940402803811F00C9475278EE991E006
:102550006EE870E00E940402803811F00C94752738
:102560008EE991E067E970E00E940402803811F082
:102570000C9475278EE991E064EA70E00E940402F1
:10258000803811F00C94752781E080931B023DE2A6
:10259000E32E32E0F32E00E010E00F5F1F4F8EE9D4
:1025A00091E0B8010E940402D7018D937D010032B1
:1025B000110599F78EE991E062E270E00E94040251
:1025C00080934E028EE991E063E270E00E94040283
:1025D00080934F0220E5E22E22E0F22E04E210E08A
:1025E0008EE991E0B8010E940402F70181937F0116
:1025F0000F5F1F4F0A32110599F796E5E92E92E019
:10260000F92E0AE210E08EE991E0B8010E9404027E
:10261000D7018C930C5F1F4F8EE991E0B8010E94A7
:102620000402F70184830C5F1F4F8EE991E0B8012B
:102630000E940402D70118968C930C5F1F4F8EE9FD
:1026400091E0B8010E940402F70184870C5F1F4FDC
:102650008EE991E0B8010E940402D70150968C9354
:102660000C5F1F4F8EE991E0B8010E940402F70150
:10267000848B035110400894E11CF11C0E321105AB
:1026800011F68EE6E82E82E0F82E02E410E08EE9E4
:1026900091E0B8010E940402D7018D937D010F5F84
:1026A0001F4F0238110599F78EE991E062E870E05A
:1026B0000E940402182F8EE991E063E870E00E9406
:1026C0000402312F20E0280F311D3093B0022093F7
:1026D000AF028EE991E065E870E00E940402809309
:1026E000B1028EE991E066E870E00E9404028093F6
:1026F000B2028EE991E067E870E00E9404028093E4
:10270000B3028EE991E068E870E00E9404028093D1
:10271000B4028EE991E06AE870E00E9404028093BE
:10272000B5028EE991E06BE870E00E9404028093AC
:10273000B6028EE991E06DE870E00E940402809399
:10274000B7028EE991E06FE870E00E940402182F52
:102750008EE991E060E970E00E940402312F20E0F0
:10276000280F311D3093B9022093B8028EE991E011
:1027700061E970E00E940402182F8EE991E062E99D
:1027800070E00E940402312F20E0280F311D3093A9
:10279000BB022093BA028EE991E063E970E00E94E7
:1027A0000402182F8EE991E064E970E00E940402AF
:1027B000312F20E0280F311D3093BD022093BC0241
:1027C0008EE991E065E970E00E940402182F8EE91D
:1027D00091E066E970E00E940402312F20E0280FAA
:1027E000311D3093BF022093BE028EE991E068E96B
:1027F00070E00E940402182F8EE991E069E970E010
:102800000E940402312F20E0280F311D3093C102B5
:102810002093C0028EE991E06AE970E00E94040210
:10282000182F8EE991E06BE970E00E940402312FCD
:1028300020E0280F311D3093C3022093C2028EE99D
:1028400091E06CE970E00E940402182F8EE991E09B
:102850006DE970E00E940402312F20E0280F311D45
:102860003093C5022093C4028EE991E06EE970E0D6
:102870000E940402182F8EE991E06FE970E00E9437
:102880000402312F20E0280F311D3093C70220931E
:10289000C6028EE991E060EA70E00E940402182FFF
:1028A0008EE991E061EA70E00E940402312F20E09D
:1028B000280F311D3093C9022093C8028EE991E0A0
:1028C00062EA70E00E940402182F8EE991E063EA48
:1028D00070E00E940402312F20E0280F311D309358
:1028E000CB022093CA028091B102882309F463C00D
:1028F00061E00E9453298091B10260E00E94732937
:102900008091B10260E00E945329FF24F39400E01B
:1029100010E08091B1020E94C029019711F0FF24BC
:1029200006C068EE73E080E090E00E9478280F5FB8
:102930001F4F0530110569F7FF20E9F100E010E0B5
:102940008EE991E0B8014FEF0E940B020F5F1F4F1D
:10295000B4E000301B07A1F78091B202882319F080
:1029600061E00E9453298091B402882319F061E04C
:102970000E9453298091B20261E00E9473298091E4
:10298000B40261E00E94732962E370E080E090E0AD
:102990000E9478288091B20260E00E9473298091A1
:1029A000B40260E00E94732962E370E080E090E08E
:1029B0000E947828DFCF8091B302882341F061E044
:1029C0000E9453298091B30260E00E947329809194
:1029D000B402882341F061E00E9453298091B4023F
:1029E00060E00E9473298091B50290E025E230E01A
:1029F000FC01E29FC001E39F900DF29F900D112416
:102A00004DB65EB6481A590A0FB6F8945EBE0FBEB0
:102A10004DBE2DB73EB72F5F3F4FCF58DD4F3983A7
:102A20002883C157D2408091B60290E026E230E080
:102A3000AC01429FC001439F900D529F900D112405
:102A40006DB77EB7681B790B0FB6F8947EBF0FBECB
:102A50006DBF8DB79EB70196CD58DD4F99838883A2
:102A6000C357D2402091B70230E0C901880F991FA7
:102A7000820F931FADB7BEB7A81BB90B0FB6F89462
:102A8000BEBF0FBEADBFEDB7FEB73196CB58DD4F21
:102A9000F983E883C557D2408F01EE24FF246901F2
:102AA0000894C11CD11C02C00E949D0FC80108944B
:102AB000E11CF11C0D5F1F4FEC14FD04A9F7CF586A
:102AC000DD4FF881C157D240C558DD4FF883CB5751
:102AD000D240CE58DD4F4880C257D240C458DD4F57
:102AE0004882CC57D2408F2F942D9C01D90120E0F1
:102AF00030E04FEF65E270E026C011964C931197DD
:102B000012964C93129714964C93149713964C93D9
:102B10001397269FF001279FF00D369FF00D11248B
:102B20003596CF58DD4F88819981C157D240E80F43
:102B3000F91F80E090E01192019680329105D9F75B
:102B40002F5F3F4F95968091B50290E02817390787
:102B5000A4F2CD58DD4F9881C357D240C358DD4F02
:102B60009883CD57D240CC58DD4FA881C457D2406E
:102B7000C258DD4FA883CE57D240892F9A2F9C018F
:102B8000D90120E030E06FEF46E250E024C06C93C2
:102B900011966C93119712961D921D921D921C9284
:102BA0001597249FF001259FF00D349FF00D1124FF
:102BB0003696CD58DD4F48805980C357D240E40D3A
:102BC000F51D80E090E01192019680329105D9F7D1
:102BD0002F5F3F4F96968091B60290E028173907F5
:102BE000B4F26091B8027091B90280E090E00E9466
:102BF000782881E090E060E020E030E040E050E0C4
:102C00000E94A71180914E02882309F448C08FE9E1
:102C100091E060E572E020E63AEE40E050E010ED31
:102C2000E12E17E0F12E012D112D0E940B090197C5
:102C3000F9F48FE991E066E572E00E9448068FE9B9
:102C400091E06AE572E00E9439068FE991E066E65C
:102C500072E00E942A068FE991E06EE572E00E9420
:102C60001B068FE991E062E672E00E940C0623C029
:102C70002091C0023091C10240E050E081E090E03C
:102C800060E00E94A7110E949F1181E090E061E046
:102C900020E030E040E050E00E94A7110CC084EC3E
:102CA00091E060E572E046E552E026E632E00AE5B2
:102CB00012E00E94A10B82E090E060E020E030E0B2
:102CC00040E050E00E94A71180914F02882309F450
:102CD00046C08E01045D1D4FC8010E949D0BC801B6
:102CE0006EE672E042E652E00E944C0AC8010E9481
:102CF000FF0AE090C202F090C3020DC06AE070E0EB
:102D000080E090E00E94782826EF3FEFE20EF31E6D
:102D10001E141F0474F4C8010E945D0A90E000971D
:102D200069F3019731F4C8016AE672E00E943D0A36
:102D300016C02091C4023091C50240E050E082E00C
:102D400090E060E00E94A7110E949F1182E090E055
:102D500061E020E030E040E050E00E94A7110E94D6
:102D60005228DC01CB010E940C2E83E090E060E051
:102D700020E030E040E050E00E94A711C090AF0298
:102D8000D090B00260E074E080E090E02EEF3BEF86
:102D900040E050E00E94EE2D8B019C017E010894E2
:102DA000E11CF11CC7016AE672E0A60198010E94CD
:102DB000E205C7010E94B005882311F40C945E2738
:102DC0000E944428C359DD4F688379838A839B839B
:102DD000CD56D240B3E72B2EB1E03B2E8DE791E0EC
:102DE000CF57DD4F8883C158D240CE57DD4F9883EF
:102DF000C258D240C101CD57DD4F2882C358D240BE
:102E0000CC57DD4F9883C458D2404BE452E04C0F6E
:102E10005D1F405E5F4FC158DD4F59834883CF57D8
:102E2000D2400C9441270E944428C359DD4F288189
:102E300039814A815B81CD56D240621B730B840B72
:102E4000950B2091CA023091CB0240E050E062170E
:102E5000730784079507A0F089E090E060E020E028
:102E600030E040E050E00E94A7110E949F1189E0ED
:102E700090E061E020E030E040E050E00E94A711E7
:102E8000C358DD4F8881CD57D240C258DD4F98815D
:102E9000CE57D2409C016901AA24BB24A6E26A2E27
:102EA000712C99249A9431C1D6018C918F3F19F1DC
:102EB000A69CF001A79CF00DB69CF00D112436964F
:102EC000CD58DD4F48805980C357D240E40DF51DE1
:102ED000DF0120E030E08C91882369F42F5F3F4FC1
:102EE000119620323105B9F70C94E427119201961E
:102EF00080329105D9F7D6018C918F3F09F4FDC03E
:102F00001296ED90FD900D911C9115970E9444280A
:102F10006E157F058007910708F4EFC00E944428D2
:102F2000F601E280F380048115816E197F09800B20
:102F3000910B61587E4E8643904008F0DEC00E949F
:102F40004428E61AF70A080B190B20E8E2162EEEC1
:102F5000F20626E3020720E0120708F4CEC0A69C82
:102F6000D001A79CB00DB69CB00D11241696CD587B
:102F7000DD4F48815981C357D240A40FB51F7D0151
:102F800060E070E091C000E010E081E090E0002E91
:102F900002C0880F991F0A94E2F7582F282F30E0BB
:102FA000F701808190E082239323181619060CF014
:102FB00070C0F6018181813039F1813020F082309A
:102FC00009F067C040C0F601808190E0F5E24F2E25
:102FD000512C849DF001859DF00D949DF00D1124E0
:102FE000CF58DD4F88819981C157D240E80FF91F32
:102FF000E60FF71F4581842F90E02823392312160E
:1030000013060CF43FC045C0F601808190E0E5E274
:103010004E2E512C849DF001859DF00D949DF00D58
:103020001124CF58DD4F88819981C157D240E80FD4
:10303000F91FE60FF71F4581842F90E028233923DD
:10304000232B39F524C0F601808190E045E2442E1F
:10305000512C849DF001859DF00D949DF00D11245F
:10306000CF58DD4F88819981C157D240E80FF91FB1
:10307000E60FF71F4581842F90E0822393231816D3
:1030800019061CF4451B458304C0892B11F4540F09
:1030900055830F5F1F4F0830110509F076CF6F5F22
:1030A0007F4F0894E11CF11CF601808190E0F5E26D
:1030B0004F2E512C849DF001859DF00D949DF00DB7
:1030C0001124CF58DD4F28813981C157D240E20FFA
:1030D000F31F808190E0681779070CF454CFF60154
:1030E00090829182128213821482158280E090E095
:1030F0001D92019680329105D9F70894A11CB11C4C
:10310000E6E24E2E512CC40CD51C8091B60290E004
:10311000A816B9060CF4C8CECF58DD4FA880B980E8
:10312000C157D24024E030E0A20EB31EC558DD4F97
:103130008881CB57D240C458DD4F9881CC57D240BC
:103140009C017901CC24DD247BC0D70111968C91A0
:10315000282F30E0C9010297089730F02E503040F8
:103160002630310508F063C0F7018281282F30E056
:10317000C9010297089730F02E50304026303105B3
:1031800008F055C0D70114968C91282F30E0C90162
:103190000297089730F02E5030402630310508F065
:1031A00046C0F701808175E2472E512CC49C8001F6
:1031B000C59C100DD49C100D1124080F111D0C5F1F
:1031C0001F4FCF58DD4F28813981C157D240020FA0
:1031D000131F0DC0D70112968C91129711966C9106
:1031E00041E0F80120810E940F2A015010400A1589
:1031F0001B0581F7D70114968C9161E00E94732919
:10320000F701848160E00E947329D70113964C91E5
:10321000242F30E0C9010297089728F02E50304043
:103220002630310520F4842F61E00E947329089430
:10323000C11CD11CE5E2F0E0EE0EFF1EAE0EBF1E7B
:103240008091B50290E0C816D9060CF47ECF7E01BD
:103250000894E11CF11CC7010E942A05892B11F476
:103260000C9441270E944428C359DD4F6883798319
:103270008A839B83CD56D240C7010E94590500978F
:10328000A9F4C7010E944A05C70161E00E94120526
:1032900086E090E060E020E030E040E050E00E9416
:1032A000A7110E949F1186E090E06AC181309105CC
:1032B00079F4C7010E944A05C70161E00E94120526
:1032C000C7016AE00E941205C7016CE172E011C0FB
:1032D0008230910591F4C7010E944A05C70161E05F
:1032E0000E941205C70160E20E941205C7016DE24B
:1032F00072E00E949C050C9441278330910509F0EF
:1033000048C1CF57DD4FF881C158D240F88BCE5716
:10331000DD4F4880C258D240498A8B819C819B8B6B
:103320008A8B8D819E819D8B8C8B8F8198859F8BC5
:103330008E8BCD57DD4F5880C358D240588ECC5716
:10334000DD4F2881C458D240298F8B858A8F8C8588
:103350009D859C8F8B8F8E859F859E8F8D8F4091B5
:10336000C8025091C90260E070E0CE0140960E9410
:103370001612C7010E945905B82ECF57DD4F38816C
:10338000C158D2403F8F48A28B819C819AA389A3C8
:103390008D819E819CA38BA38F8198859EA38DA3F5
:1033A0005FA2CC57DD4F4881C458D24048A78B85D7
:1033B00089A78C859D859BA78AA78E859F859DA7BC
:1033C0008CA74091C8025091C90260E070E0CE0124
:1033D0004F960E941612C7010E945905182FCF5709
:1033E000DD4F5881C158D2405EA74FA68B819C818A
:1033F00099AB88AB8D819E819BAB8AAB8F81988581
:103400009DAB8CAB5EAACC57DD4F6881C458D240CF
:103410006FAB8B8588AF8C859D859AAF89AF8E8584
:103420009F859CAF8BAF4091C8025091C90260E06C
:1034300070E0CE018E960E941612C7010E945905B7
:10344000C82ECF57DD4F7881C158D2407DAF4EAEE8
:103450008B819C81FE01FF96918380838D819E816B
:10346000FE01EF5BFF4F918380838F819885FE0182
:10347000ED5BFF4F91838083FE01EB5BFF4F318259
:1034800020828B85FE01E95BFF4F80838C859D85C3
:10349000FE01E85BFF4F918380838E859F85FE014F
:1034A000E65BFF4F918380834091C8025091C9022F
:1034B00060E070E0CE01CD960E941612C7010E9416
:1034C0005905D82EFE01E45BFF4F8DE791E0918313
:1034D00080838B819C81938382838D819E81958360
:1034E00084838F819885978386835086CC57DD4F60
:1034F0009881C458D24091878B8582878C859D8521
:10350000948783878E859F85968785874091C8029B
:103510005091C90260E070E0CF010E941612C7010D
:103520000E945905082FC7010E944A05C70161E0A2
:103530000E94120560E0113009F461E0C858DD4FC7
:10354000C882C857D240C958DD4F1882C757D240E9
:10355000C958DD4F28813981C757D2402D0D311D03
:10356000442737FD4095542F8B2D90E00E94A711E2
:10357000013011F00C9441270E949F118B2D90E097
:1035800061E020E030E040E050E00E94A7110C94A0
:10359000412784309105D1F4C7010E944A050E9459
:1035A000810F8C0197FF02C00C94F327C70161E0E3
:1035B0000E941205612F772767FD7A95C7010E9447
:1035C00012051070C701602F0C943F2785309105BC
:1035D000A9F4C7010E944A058091B402882311F41E
:1035E0000C94792661E00E9473296AE070E080E023
:1035F00090E00E9478288091B40224C2873091051F
:1036000009F09EC0C7010E944A05C70161E00E94FF
:103610001205C70160914E020E94120500E512E0FA
:10362000C701FE2CE92E8F2D9E2DD8016D918D01A5
:103630000E941205B2E006351B07A9F78F2D9E2DBB
:10364000F80160810E9412058F2D9E2DD8011196E0
:103650006C910E9412058F2D9E2DF80162810E94AF
:1036600012058F2D9E2DD80113966C910E94120584
:103670008F2D9E2DF80164810E9412058F2D9E2DA5
:10368000D80115966C910E9412058F2D9E2DF80180
:1036900066810E9412058F2D9E2DD80117966C9180
:1036A0000E9412058F2D9E2DF80160850E94120543
:1036B0008F2D9E2DD80119966C910E9412058F2D89
:1036C0009E2DF80162850E9412058F2D9E2DD80136
:1036D0001B966C910E9412058F2D9E2DF80164851A
:1036E0000E9412058F2D9E2DD8011D966C910E946F
:1036F00012058F2D9E2DF80166850E9412058F2DD3
:103700009E2DD8011F966C910E9412058F2D9E2D23
:10371000F80160890E9412058F2D9E2DD8015196C7
:103720006C910E9412058F2D9E2DF80162890E94D6
:1037300012058F2D9E2DD80153966C910C943F2726
:103740008830910509F58E010F5F1F4FC8010E9457
:103750004A05C80161E00E941205EE24FF24D02E24
:10376000012F8EE991E0B7010E940402682F8D2D90
:10377000902F0E9412050894E11CF11CB5EAEB168B
:10378000F10479F70C9441278930910509F05CC068
:1037900000E010E07E010894E11CF11CCF57DD4FE2
:1037A000E881C158D2406C96EFAF6C97CE57DD4F91
:1037B000F881C258D2406D96FFAF6D978B819C8186
:1037C0006F969FAF8EAF6F978D819E81A1969FAFB1
:1037D0008EAFA1978F819885A3969FAF8EAFA39749
:1037E000A5963FAE2EAEA5978B85A6968FAFA697D2
:1037F0008C859D85A8969FAF8EAFA8978E859F8557
:10380000AA969FAF8EAFAA974091C8025091C90265
:1038100060E070E0CE01855A9F4F0E941612C701EA
:103820000E945905482F8EE991E0B8010E940B02D1
:103830000F5F1F4F053A110509F0B0CFC7010E9475
:103840004A05C7010C947B268A30910509F07FC098
:10385000FE01E659FF4F5DE7452E51E0552E51829E
:1038600040828B819C81938382838D819E8195830D
:1038700084838F81988597838683318620868B8584
:1038800082878C859D85948783878E859F85968783
:1038900085874091C8025091C90260E070E0CF0175
:1038A0000E9416128E010F5F1F4FC8010E9459051A
:1038B0007C01FE01E758FF4F518240828B819C8141
:1038C000938382838D819E81958384838F81988564
:1038D00097838683318620868B8582878C859D851C
:1038E000948783878E859F85968785874091C802B8
:1038F0005091C90260E070E0CF010E941612C80129
:103900000E9459056C01C8010E944A059701C70130
:103910000297089738F02E5030402630310510F0CD
:103920000C943C27D7FE02C00C943C2722E0C21620
:10393000D10414F00C943C27CD2819F48E2D60E0AE
:1039400002C08E2D61E00E9453290C9479268B30A1
:10395000910509F07FC0FE01E857FF4F4DE751E0A8
:10396000518340838B819C81938382838D819E814F
:10397000958384838F81988597838683318620867B
:103980008B8582878C859D85948783878E859F858F
:10399000968785874091C8025091C90260E070E027
:1039A000CF010E9416128E010F5F1F4FC8010E94A7
:1039B00059057C01FE01E956FF4F6DE771E0718307
:1039C00060838B819C81938382838D819E8195838B
:1039D00084838F81988597838683318620868B8523
:1039E00082878C859D85948783878E859F85968722
:1039F00085874091C8025091C90260E070E0CF0114
:103A00000E941612C8010E9459056C01C8010E944B
:103A10004A059701C7010297089738F02E503040A9
:103A20002630310510F00C943C27D7FE02C00C94D0
:103A30003C2772E0C716D10414F00C943C27CD2823
:103A400019F48E2D60E002C08E2D61E00E94732972
:103A50000C9479268C30910509F071C0FE01EA556D
:103A6000FF4F8DE791E0918380838B819C819383CD
:103A700082838D819E81958384838F8198859783AE
:103A80008683318620868B8582878C859D85948769
:103A900083878E859F85968785874091C802509140
:103AA000C90260E070E0CF010E9416126E01089416
:103AB000C11CD11CC6010E9459058C01FE01EB54AA
:103AC000FF4FADE7B1E0B183A0838B819C819383ED
:103AD00082838D819E81958384838F81988597834E
:103AE0008683318620868B8582878C859D85948709
:103AF00083878E859F85968785874091C8025091E0
:103B0000C90260E070E0CF010E941612C6010E9457
:103B100059057C01C6010E944A050330110531F0A8
:103B20000530110519F00630110531F4802FB70169
:103B30000E94FA280C947926C6010C943E278D30F9
:103B4000910509F05DC0FE01EC53FF4F4DE7442E97
:103B500041E0542E518240828B819C8193838283E9
:103B60008D819E81958384838F81988597838683B9
:103B7000318620868B8582878C859D859487838777
:103B80008E859F85968785874091C8025091C9028E
:103B900060E070E0CF010E9416127E010894E11CE3
:103BA000F11CC7010E9459058C01C7010E944A05FA
:103BB0009801C8010297089738F02E5030402630FF
:103BC000310510F00C94F327802F0E94C029019733
:103BD00049F48E010F5F1F4FC80161E00E9412057A
:103BE0000C94EE25802F0E94C0298E010F5F1F4F7D
:103BF000892B09F01EC6C80161E00E94120519C692
:103C00008E30910509F06AC0FE01ED52FF4F2DE79D
:103C100031E0318320838B819C81938382838D81EA
:103C20009E81958384838F8198859783868331864F
:103C300020868B8582878C859D85948783878E855A
:103C40009F85968785874091C8025091C90260E0A0
:103C500070E0CF010E9416128E010F5F1F4FC80146
:103C60000E9459056C01C8010E944A05C6010297CD
:103C7000089730F0C6010E97069710F00C943C2779
:103C80003EE0C316D10414F40C943C277E01089442
:103C9000E11CF11CC70161E00E94120586010E5073
:103CA0001040802F0E94DC286AE070E080E090E005
:103CB0000E947828802F0E94DC288C0160E071E04F
:103CC0000E943F2EC7010E941205C80160E071E00A
:103CD0000E943F2E682FC7010C943F278431910525
:103CE00009F0C5C1FE01EE51FF4F4DE751E0518390
:103CF00040838B819C81938382838D819E81958378
:103D000084838F81988597838683318620868B85EF
:103D100082878C859D85948783878E859F859687EE
:103D200085874091C8025091C90260E070E0CF01E0
:103D30000E9416128E010F5F1F4FC8010E94590585
:103D40005C01FE01EF50FF4F6DE771E0718360830E
:103D50008B819C81938382838D819E8195838483D3
:103D60008F81988597838683318620868B8582878D
:103D70008C859D85948783878E859F85968785878B
:103D80004091C8025091C90260E070E0CF010E94EA
:103D90001612C8010E9459057C01FE01E050FF4F38
:103DA0008DE791E0918380838B819C8193838283D3
:103DB0008D819E81958384838F8198859783868367
:103DC000318620868B8582878C859D859487838725
:103DD0008E859F85968785874091C8025091C9023C
:103DE00060E070E0CF010E941612C8010E945905E0
:103DF000682E592EFE01E15FFE4FADE7B1E0B183C1
:103E0000A0838B819C81938382838D819E81958306
:103E100084838F81988597838683318620868B85DE
:103E200082878C859D85948783878E859F859687DD
:103E300085874091C8025091C90260E070E0CF01CF
:103E40000E941612C8010E945905982E792EFE0173
:103E5000E25EFE4F2DE731E0318320838B819C8130
:103E6000938382838D819E81958384838F819885BE
:103E700097838683318620868B8582878C859D8576
:103E8000948783878E859F85968785874091C80212
:103E90005091C90260E070E0CF010E941612C80183
:103EA0000E945905882EFE01E35DFE4F4DE751E06B
:103EB000518340838B819C81938382838D819E81FA
:103EC000958384838F819885978386833186208626
:103ED0008B8582878C859D85948783878E859F853A
:103EE000968785874091C8025091C90260E070E0D2
:103EF000CF010E941612C8010E9459056C01C80129
:103F00000E944A059701C7010297089730F02E508A
:103F100030402630310508F0AFC7262D352DC901B8
:103F20000297089730F02E5030402630310508F0C7
:103F3000A3C7292D372DC9010297089730F02E50BD
:103F400030402630310508F097C7B7FC95C78091FF
:103F5000B50290E08A159B050CF48EC71C141D0455
:103F60000CF08AC751E2C516D1040CF085C765E292
:103F700070E0A69E8001A79E100DB69E100D112424
:103F8000CF58DD4F88819981C157D240080F191F42
:103F9000D8011196EC92119712966C921297149682
:103FA0009C92149713968C921397CC928E2D61E06D
:103FB0000E945329F801818160E00E947329D80191
:103FC00012968C9161E00E945329F801828160E091
:103FD0000E947329D80114968C9161E00E945329A4
:103FE000F801848160E00E947329D80113964C91F6
:103FF000242F30E0C9010297089728F02E50304056
:1040000026303105D0F4842F61E00E94532935E237
:10401000432E512CA49CF001A59CF00DB49CF00DF6
:104020001124CF58DD4F28813981C157D240E20F8A
:10403000F31F838160E00E94732945E250E0A49E53
:10404000F001A59EF00DB49EF00D11243596CF58C9
:10405000DD4F68817981C157D240E60FF71F80E0BC
:1040600090E01192019680329105D9F742C68531D0
:10407000910509F0F7C0FE01E45CFE4F8DE791E089
:10408000918380838B819C81938382838D819E81A8
:10409000958384838F819885978386833186208654
:1040A0008B8582878C859D85948783878E859F8568
:1040B000968785874091C8025091C90260E070E000
:1040C000CF010E9416128E010F5F1F4FC8010E9480
:1040D0005905982E8091B502891508F4A7C3892D3A
:1040E00090E0DC01E5E2F0E0AE9FC001AF9F900DF3
:1040F000BE9F900D11240596CF58DD4FA880B98042
:10410000C157D240A80EB91E2BEFC22E2FEFD22ED0
:10411000C80ED91EEE24FF24CF58DD4F48805980A9
:10412000C157D240C40CD51C50C02DE731E0C55B4F
:10413000DE4F39832883CB54D1408B819C81C35B74
:10414000DE4F99838883CD54D1408D819E81C15BA0
:10415000DE4F99838883CF54D1408F819885CF5A81
:10416000DE4F99838883C155D140CD5ADE4F3982C5
:104170002882C355D1408B85CB5ADE4F8883C555E5
:10418000D1408C859D85CA5ADE4F99838883C65558
:10419000D1408E859F85C85ADE4F99838883C85544
:1041A000D1404091C8025091C90260E070E0CE0158
:1041B000855B9E4F0E941612C8010E945905D501C9
:1041C0008D935D010894E11CF11CF601808190E063
:1041D000E816F9060CF4A9CFC358DD4F8881CD57F6
:1041E000D240C258DD4F9881CE57D2409C01D901B0
:1041F00020E030E06FEF46E250E027C08C91891557
:1042000009F56C9311966C93119712961D921D925D
:104210001D921C921597249FF001259FF00D349F4D
:10422000F00D11243696CD58DD4F48805980C35784
:10423000D240E40DF51D80E090E0119201968032AD
:104240009105D9F72F5F3F4F96968091B60290E087
:10425000281739079CF28E010F5F1F4FC8010E947B
:104260004A05BCC48631910509F0E5C2FE01E65A53
:10427000FE4F2DE731E0318320838B819C81938336
:1042800082838D819E81958384838F819885978396
:104290008683318620868B8582878C859D85948751
:1042A00083878E859F85968785874091C802509128
:1042B000C90260E070E0CF010E9416126E010894FE
:1042C000C11CD11CC6010E945905482EFE01E759A8
:1042D000FE4F4DE751E0518340838B819C81938356
:1042E00082838D819E81958384838F819885978336
:1042F0008683318620868B8582878C859D859487F1
:1043000083878E859F85968785874091C8025091C7
:10431000C90260E070E0CF010E941612C6010E943F
:104320005905582EFE01E858FE4F6DE771E0718384
:1043300060838B819C81938382838D819E81958311
:1043400084838F81988597838683318620868B85A9
:1043500082878C859D85948783878E859F859687A8
:1043600085874091C8025091C90260E070E0CF019A
:104370000E941612C6010E945905E82EFE01E95757
:10438000FE4F8DE791E0918380838B819C819383A5
:1043900082838D819E81958384838F819885978385
:1043A0008683318620868B8582878C859D85948740
:1043B00083878E859F85968785874091C802509117
:1043C000C90260E070E0CF010E941612C6010E948F
:1043D0005905B82EFE01EA56FE4FADE7B1E0B183B4
:1043E000A0838B819C81938382838D819E81958321
:1043F00084838F81988597838683318620868B85F9
:1044000082878C859D85948783878E859F859687F7
:1044100085874091C8025091C90260E070E0CF01E9
:104420000E941612C6010E945905FF2400E010E008
:104430008701FF24EE24E80EF11C011D111DC65852
:10444000DD4FB882CA57D240C758DD4F1882C957CE
:10445000D240C758DD4FE881F981C957D240CF011A
:10446000A0E0B0E0E80EF91E0A1F1B1FFE01E55B8D
:10447000FD4F1192C158DD4F28813981CF57D2406D
:10448000E217F307B1F7E114F1040105110519F47E
:104490006624639419C08091B602482F50E0CD582D
:1044A000DD4FE881F981C357D240662420E030E037
:1044B00008C080818F3F11F4662463942F5F3F4FC3
:1044C000B69624173507ACF38091B502841508F42D
:1044D000AAC1442D50E0C559DD4F59834883CB56BE
:1044E000D24065E270E0469FC001479F900D569F05
:1044F000900D11240596CF58DD4FC880D980C15743
:10450000D240C80ED91EBBEF8B2EBFEF9B2E880E5C
:10451000991EAA24BB24CF58DD4F88819981C157A9
:10452000D240880E991ECBC0ADE7B1E0CB55DE4F2F
:10453000B983A883C55AD1408B819C81C955DE4F70
:1045400099838883C75AD1408D819E81C755DE4F9C
:1045500099838883C95AD1408F819885C555DE4F8C
:1045600099838883CB5AD140C355DE4F3982288244
:10457000CD5AD1408B85C155DE4F8883CF5AD1406B
:104580008C859D85C055DE4F99838883C05BD14063
:104590008E859F85CE54DE4F99838883C25BD14040
:1045A0004091C8025091C90260E070E0CE018B5585
:1045B0009E4F0E941612CE0101960E945905782E38
:1045C000662009F46FC060E070E0E82FF0E081E061
:1045D00090E0062E02C0880F991F0A94E2F7582F28
:1045E000282F30E0C9018E239F231816190674F571
:1045F000B1E05B1681F05B1620F042E0541631F515
:1046000014C0D6014C91842F90E028233923121630
:104610001306A4F01BC0D6014C91842F90E02823F0
:104620003923232B99F4540F10C0D6014C91842FB9
:1046300090E082239323181619061CF4451B4C9313
:1046400005C0892B19F4540FD6015C936F5F7F4F1F
:104650006830710509F0BBCFCD58DD4FA881B98115
:10466000C357D240E6E0F0E0AE0EBF1EFD01EA0DFA
:10467000FB1D2AEF3FEFA20EB31E20E030E0472DD6
:1046800040950AC08C91841519F48081842380831D
:104690002F5F3F4F9696B6968091B60290E028170E
:1046A000390784F3EBE4F2E0EC0FFD1FEA0DFB1D8C
:1046B00070820894A11CB11C0894C11CD11CD401A7
:1046C0008C9190E0A816B9060CF42ECF662009F460
:1046D000A1C0E114F1040105110509F49BC00E9479
:1046E00044289B01AC012E0D3F1D401F511F211579
:1046F00031054105510521F421E030E040E050E072
:104700008091B602A82FB0E0CD58DD4FE881F98145
:10471000C357D24060E070E079C08081B6968F3F89
:1047200009F072C086E290E0689FF001699FF00D89
:10473000789FF00D1124CD58DD4F88819981C357A2
:10474000D240E80FF91F4082552019F481E081839F
:1047500006C092E0591611F4518201C0118283E122
:1047600090E0689FF001699FF00D789FF00D112493
:104770003196EE0FFF1FCD58DD4FA881B981C35789
:10478000D240EA0FFB1F208331834283538386E2AA
:1047900090E0689FD001699FB00D789FB00D112403
:1047A0001696CD58DD4FE881F981C357D240AE0F40
:1047B000BF1F20E030E0C559DD4F48805980CB56FF
:1047C000D24065E270E0469EA001479E500D569E85
:1047D000500D1124CF58DD4F88819981C157D240A7
:1047E000480F591F0AC0EBE4F2E0EC0FFD1FE20F87
:1047F000F31F80818D932F5F3F4FFA01808190E0FE
:104800002817390784F306C06F5F7F4F6A177B074D
:104810000CF483CF8E010F5F1F4FC8010E944A0521
:10482000662039F0DBC18E010F5F1F4FC8010E9467
:104830004A05C80123C38E31910509F0C1C0FE01AC
:10484000EC54FE4F5DE7452E51E0552E51824082DB
:104850008B819C81938382838D819E8195838483C8
:104860008F81988597838683318620868B85828782
:104870008C859D85948783878E859F859687858780
:104880004091C8025091C90260E070E0CF010E94DF
:1048900016127E010894E11CF11CC7010E94590503
:1048A0008C01C7010E944A050B30110508F09BC31B
:1048B0000530110509F454C006301105B4F4023076
:1048C0001105C9F10330110544F40115110529F151
:1048D0000130110509F06FC027C00330110591F1B7
:1048E0000430110509F067C034C00830110509F41F
:1048F0004CC00930110544F406301105C1F10730F0
:10490000110509F058C03AC00930110509F444C036
:104910000A30110509F04FC046C089E593E04CE22A
:1049200051E060E070E045C089E593E040EB54E081
:1049300060E070E03EC089E593E040E659E060E069
:1049400070E037C089E593E040EC52E160E070E050
:1049500030C089E593E040E855E260E070E029C0AE
:1049600089E593E040E458E360E070E022C089E527
:1049700093E040E05BE460E070E01BC089E593E019
:1049800040E850E760E070E014C089E593E040E063
:1049900056E960E070E00DC089E593E040E051EE3B
:1049A00060E070E006C089E593E040E052EC61E031
:1049B00070E00E948D2A89E593E00E94C22B99C184
:1049C0008F31910509F096C0FE01ED53FE4F2DE7A2
:1049D00031E0318320838B819C81938382838D811D
:1049E0009E81958384838F81988597838683318682
:1049F00020868B8582878C859D85948783878E858D
:104A00009F85968785874091C8025091C90260E0D2
:104A100070E0CF010E9416128E010F5F1F4FC80178
:104A20000E945905CC24DD2476014C01AA24BB2424
:104A300056C04DE751E0CE52DE4F59834883C25DE8
:104A4000D1408B819C81CC52DE4F99838883C45D99
:104A5000D1408D819E81CA52DE4F99838883C65D85
:104A6000D1408F819885C852DE4F99838883C85D75
:104A7000D140C652DE4F39822882CA5DD1408B8533
:104A8000C452DE4F8883CC5DD1408C859D85C35256
:104A9000DE4F99838883CD5DD1408E859F85C1523D
:104AA000DE4F99838883CF5DD1404091C8025091F9
:104AB000C90260E070E0CE018E529E4F0E94161235
:104AC000C8010E945905682F89E593E040E050E055
:104AD0000E940A2D0894C11CD11CE11CF11CC814B1
:104AE000D904EA04FB0408F4A4CFC8010E944A05D3
:104AF000C80101C18032910509F063C0FE01EF5188
:104B0000FE4F6DE771E0718360838B819C8193839D
:104B100082838D819E81958384838F8198859783FD
:104B20008683318620868B8582878C859D859487B8
:104B300083878E859F85968785874091C80250918F
:104B4000C90260E070E0CF010E9416128E010F5F73
:104B50001F4FC8010E9459057C01C8010E944A05E7
:104B6000C80161E00E941205C8016E2D0E94120565
:104B700055245394AA24BB24650137018824992421
:104B8000F02E012F18C0552009F42FC289E593E0BB
:104B90000E94862B882309F428C289E593E00E94AD
:104BA0009A2B682F8F2D902F0E9412050894A11C1C
:104BB000B11CC11CD11CA614B704C804D90418F335
:104BC00060C18132910561F48E010F5F1F4FC801F2
:104BD0000E944A0589E593E00E94C22BC8018BC060
:104BE0008832910509F089C0FE01E051FE4F8DE742
:104BF00091E0918380838B819C81938382838D81DB
:104C00009E81958384838F8198859783868331865F
:104C100020868B8582878C859D85948783878E856A
:104C20009F85968785874091C8025091C90260E0B0
:104C300070E0CF010E9416128E010F5F1F4FC80156
:104C40000E9459057C01FE01E150FE4FADE7B1E045
:104C5000B183A0838B819C81938382838D819E818C
:104C6000958384838F819885978386833186208678
:104C70008B8582878C859D85948783878E859F858C
:104C8000968785874091C8025091C90260E070E024
:104C9000CF010E941612C8010E945905D82EC92EB4
:104CA000C8010E944A05F7FCE7C08091B70290E076
:104CB000E816F9060CF0E0C02D2D3C2DC901029735
:104CC000089730F02E5030402630310508F0D4C01F
:104CD000C701880F991F8E0D9F1DCB58DD4FE881AE
:104CE000F981C557D2408E0F9F1F6D2D7C2D0E94DC
:104CF000DA10CE01019661E0C2C0899709F0C1C007
:104D00003DE7432E31E0532EC25FDD4F598248828A
:104D1000CE50D2408B819C81C05FDD4F99838883C8
:104D2000C051D2408D819E81CE5EDD4F99838883B4
:104D3000C251D2408F819885CC5EDD4F99838883A4
:104D4000C451D240CA5EDD4F39822882C651D2405A
:104D50008B85C85EDD4F8883C851D2408C859D8588
:104D6000C75EDD4F99838883C951D2408E859F8568
:104D7000C55EDD4F99838883CB51D2404091C802F4
:104D80005091C90260E070E0CE01825F9D4F0E94A9
:104D900016126E010894C11CD11CC6010E9459054F
:104DA0007C01C35EDD4F59824882CD51D2408B8158
:104DB0009C81C15EDD4F99838883CF51D2408D8124
:104DC0009E81CF5DDD4F99838883C152D2408F8110
:104DD0009885CD5DDD4F99838883C352D240CB5DEA
:104DE000DD4F39822882C552D2408B85C95DDD4FA7
:104DF0008883C752D2408C859D85C85DDD4F9983DD
:104E00008883C852D2408E859F85C65DDD4F9983C9
:104E10008883CA52D2404091C8025091C90260E0D2
:104E200070E0CE01835E9D4F0E941612C6010E9463
:104E300059058C01C6010E944A05F7FC1DC08091EE
:104E4000B70290E0E816F906BCF417FD15C0053B63
:104E5000110594F4C701880F991F8E0D9F1DCB5823
:104E6000DD4F28813981C557D240820F931FB80189
:104E70000E94F30FC6013FCFCE01019660E00E9471
:104E80001205CE0101960E942E05882311F00C9484
:104E9000131789E090E060E020E030E040E050E06F
:104EA0000E94A7110E949F1189E090E061E020E03C
:104EB00030E040E050E00E94A71116C02091C602E9
:104EC0003091C70240E050E083E090E060E00E9453
:104ED000A7110E949F1183E090E061E020E030E0A4
:104EE00040E050E00E94A711FFCF10921B028DE21C
:104EF00092E061E271E00E94FD0181E080934E0248
:104F000080934F028EED809350028DEA8093510280
:104F10008EEB809352028FEE809353028FEF80933B
:104F20005402809355028EE692E062E471E00E94A2
:104F3000FD0185E390E09093B0028093AF0298E08A
:104F40009093B1028DE08093B20289E08093B30226
:104F50009093B4021092B5021092B6021092B7026A
:104F600028E833E13093B9022093B80284E690E058
:104F70009093BB028093BA0288EC90E09093BD02BC
:104F80008093BC0284EF91E09093BF028093BE02B5
:104F90003093C1022093C0023093C3022093C20217
:104FA00080E197E29093C5028093C40220E23EE440
:104FB0003093C7022093C60288EE93E09093C90213
:104FC0008093C8020C946F14D6019C9211969C9207
:104FD000119712961D921D921D921C92159780E0BA
:104FE00090E00C947617C70149CF8F2D902F60E089
:104FF0000E9412055524DACD1F920F920FB60F9220
:1050000011242F933F938F939F93AF93BF938091DE
:10501000D0029091D102A091D202B091D3023091EE
:10502000D4020196A11DB11D232F2D5F2D3720F035
:105030002D570196A11DB11D2093D4028093D0025B
:105040009093D102A093D202B093D3028091CC026C
:105050009091CD02A091CE02B091CF020196A11DF8
:10506000B11D8093CC029093CD02A093CE02B09359
:10507000CF02BF91AF919F918F913F912F910F9050
:105080000FBE0F901F9018958FB7F8942091D00203
:105090003091D1024091D2025091D3028FBFB90119
:1050A000CA0108959FB7F8942091CC023091CD02A7
:1050B0004091CE025091CF0286B5A89B06C08F3F8B
:1050C00021F02F5F3F4F4F4F5F4F9FBF542F432F14
:1050D000322F2227280F311D411D511D82E0220F42
:1050E000331F441F551F8A95D1F7B901CA0108958E
:1050F000EF92FF920F931F937B018C018FB7F8946F
:105100004091D0025091D1026091D2027091D302AD
:105110008FBF2FB7F8948091D0029091D102A091C7
:10512000D202B091D3022FBF841B950BA60BB70BF5
:10513000E816F9060A071B0760F71F910F91FF9009
:10514000EF900895789484B5826084BD84B58160C1
:1051500084BD85B5826085BD85B5816085BDEEE67F
:10516000F0E0808181608083E1E8F0E0808182600E
:105170008083808181608083E0E8F0E080818160CD
:105180008083E1EBF0E0808184608083E0EBF0E0FD
:10519000808181608083EAE7F0E0808184608083A1
:1051A000808182608083808181608083808180684B
:1051B00080831092C1000895877090916E0192953E
:1051C000990F990F907C982B90937C0080917A0096
:1051D000806480937A0080917A0086FDFCCF2091D4
:1051E000780040917900942F80E030E0282B392B13
:1051F000C90108951F93CF93DF93182FEB0161E04E
:105200000E945329E12FF0E0E255FF4F8491833053
:1052100051F480918000806880938000D093890051
:10522000C09388003CC0843051F48091800080623B
:1052300080938000D0938B00C0938A0030C081306F
:1052400039F4209729F184B5806884BDC7BD27C093
:10525000823039F42097E1F084B5806284BDC8BD06
:105260001EC0863041F48091B00080688093B00009
:10527000C093B30014C0873041F48091B0008062C5
:105280008093B000C093B4000AC0C038D1051CF4AC
:10529000812F60E002C0812F61E00E947329DF91BD
:1052A000CF911F910895282F30E0C90186569F4F56
:1052B000FC0194912A573F4FF9018491882391F082
:1052C000E82FF0E0EE0FFF1FE859FF4FA591B491D2
:1052D000662329F48C91909589238C9308958C9161
:1052E000892B8C930895482F50E0CA0182559F4F17
:1052F000FC012491CA0186569F4FFC0194914A57A4
:105300005F4FFA0134913323D1F1222331F123305D
:1053100021F4809180008F7705C0243031F4809192
:1053200080008F7D8093800018C0213019F484B5EF
:105330008F7704C0223021F484B58F7D84BD0DC0E9
:10534000263021F48091B0008F7705C0273029F4F2
:105350008091B0008F7D8093B000E32FF0E0EE0FDE
:10536000FF1FEE58FF4FA591B491662329F48C914D
:10537000909589238C9308958C91892B8C93089513
:10538000682F70E0CB0182559F4FFC012491CB0127
:1053900086569F4FFC0144916A577F4FFB019491C1
:1053A000992319F420E030E038C0222331F1233072
:1053B00021F4809180008F7705C0243031F48091F2
:1053C00080008F7D8093800018C0213019F484B54F
:1053D0008F7704C0223021F484B58F7D84BD0DC049
:1053E000263021F48091B0008F7705C0273029F452
:1053F0008091B0008F7D8093B000892F90E0880F5E
:10540000991F84589F4FFC01A591B4918C9120E085
:1054100030E0842311F021E030E0C9010895BF920B
:10542000CF92DF92EF92FF920F931F93CF93DF9370
:10543000E82EF62EB42EC0E0D0E0022F10E087E078
:10544000C82ED12CBB2041F4B8010C2E02C075959A
:1054500067950A94E2F70AC0B6016C1B7D0BC80180
:1054600002C0959587956A95E2F7BC0161708E2D13
:105470000E9473298F2D61E00E9473298F2D60E0B7
:105480000E9473292196C830D105E1F6DF91CF91B2
:105490001F910F91FF90EF90DF90CF90BF900895F4
:1054A0001F920F920FB60F9211242F933F934F9399
:1054B0005F936F937F938F939F93AF93BF93EF937C
:1054C000FF934091C600E0915503F0915603CF0140
:1054D000019660E870E00E943F2E9C018091570386
:1054E000909158032817390739F0EB52FD4F40834C
:1054F0003093560320935503FF91EF91BF91AF91E5
:105500009F918F917F916F915F914F913F912F91DB
:105510000F900FBE0F901F9018955F926F927F9221
:105520008F929F92AF92BF92CF92DF92EF92FF92B3
:105530000F931F93CF93DF93EC013A014B0141345A
:1055400082E458078FE0680780E078070CF07FC09E
:1055500060E874E88EE190E0A40193010E94742E4B
:105560002150304040405040CA01B90122E030E0B3
:1055700040E050E00E94742E59016A01A601950195
:10558000209530954095509594E0220F331F441F8D
:10559000551F9A95D1F760E074E284EF90E00E9485
:1055A000742ECA01B9012FEF30E040E050E00E94B4
:1055B000142EA40193010E94742EC90181509F4FA3
:1055C000181619061CF4522E5A9403C055245394ED
:1055D000521A60E079E08DE390E0A40193010E940B
:1055E000742E2150304040405040CA01B90122E0A1
:1055F00030E040E050E00E94742E209530954095B8
:10560000509583E0220F331F441F551F8A95D1F711
:1056100060E074E284EF90E00E94742ECA01B90148
:105620002FEF30E040E050E00E94142EA4019301DF
:105630000E94742EC90181509F4F181619061CF440
:10564000822F815002C081E0821B851500F5E8851C
:10565000F98581E090E00A8802C0880F991F0A94BA
:10566000E2F7808360E079E08DE390E0A4019301AC
:105670000E94742E2150304040405040CA01B90170
:1056800022E030E040E050E00E94742E04C0E88543
:10569000F98510829501EC81FD813083EE81FF81D7
:1056A0002083EA85FB85208141E050E0CA010E8419
:1056B00002C0880F991F0A94E2F7282B2083EA85FD
:1056C000FB852081CA010F8402C0880F991F0A94AC
:1056D000E2F7282B2083EA85FB858081088802C0B9
:1056E000440F551F0A94E2F7842B8083DF91CF91FA
:1056F0001F910F91FF90EF90DF90CF90BF90AF90F0
:105700009F908F907F906F905F900895DC0112962C
:10571000ED91FC911397E058FF4F81919191805842
:105720009F4F20813181821B930B60E870E00E94C3
:105730003F2E0895CF93DF93DC011296ED91FC91FB
:105740001397EF01CE57DF4F48815981E058FF4F43
:1057500080819181E058F0408417950719F42FEF6C
:105760003FEF0CC0E40FF51F2081CA01019660E8ED
:1057700070E00E943F2E9983888330E0C901DF9159
:10578000CF910895DC011296ED91FC911397EE579D
:10579000FF4F80819181929382930895FC01A085AF
:1057A000B18521898C9190E0022E02C09595879554
:1057B0000A94E2F780FFF6CF0484F585E02D60833C
:1057C000089588E991E090935A038093590385EDF9
:1057D00092E090935C0380935B0385EC90E0909360
:1057E0005E0380935D0384EC90E09093600380936C
:1057F0005F0380EC90E0909362038093610381ECFF
:1058000090E0909364038093630386EC90E0909320
:1058100066038093650384E08093670383E080934D
:10582000680387E08093690385E080936A0381E0E1
:1058300080936B0308950E94A2280E949E110E94EB
:105840005312FDCF0F931F93CF93DF938C01EB0186
:1058500009C02196D801ED91FC910190F081E02DD5
:10586000C801099568816623A1F7DF91CF911F9147
:105870000F910895EF92FF920F931F93CF93DF93B1
:105880008C017B01EA010CC0D7016D917D01D8012B
:10589000ED91FC910190F081E02DC80109952197CF
:1058A000209791F7DF91CF911F910F91FF90EF908B
:1058B0000895DC01ED91FC910280F381E02D0995C2
:1058C00008952F923F924F925F926F927F928F92A4
:1058D0009F92AF92BF92CF92DF92EF92FF920F937F
:1058E0001F93DF93CF93CDB7DEB7A0970FB6F89491
:1058F000DEBF0FBECDBF1C016A017B014115510502
:105900006105710549F440E350E060E070E020E09B
:1059100030E00E941C2D56C0882499245401422E48
:1059200055246624772401E010E00C0F1D1F080D9C
:10593000191DC701B601A30192010E94522EF80160
:1059400060830894811C911CA11CB11CC701B60185
:10595000A30192010E94522EC901DA016C017D015E
:10596000C114D104E104F104F1F681E0E82EF12C38
:10597000EC0EFD1EE80CF91C3E010894611C711C24
:10598000D501C4010197A109B1096C01C818D90852
:1059900016C0F601EE0DFF1D40814A3010F4405D47
:1059A00001C0495C552747FD5095652F752FC101F2
:1059B00020E030E00E941C2D0894E108F1086E14EC
:1059C0007F0439F7A0960FB6F894DEBF0FBECDBFA7
:1059D000CF91DF911F910F91FF90EF90DF90CF90CB
:1059E000BF90AF909F908F907F906F905F904F90FF
:1059F0003F902F900895DC012115310541F4ED9180
:105A0000FC910190F081E02D642F099508950E948A
:105A1000612C0895EF92FF920F931F939A01E62E47
:105A2000FF2400E010E0B801A7010E94FB2C1F91A9
:105A30000F91FF90EF900895EF92FF920F931F93B5
:105A4000CF93DF93EC017A018B012115310541F4ED
:105A5000E881F9810190F081E02D642F09951BC048
:105A60002A303105B1F477FF10C04DE250E060E01C
:105A700070E020E030E00E941C2D10950095F0941D
:105A8000E094E11CF11C011D111DCE01B801A7011C
:105A90002AE00E94612CDF91CF911F910F91FF901E
:105AA000EF9008950F931F938C014DE050E060E05C
:105AB00070E020E030E00E941C2DC8014AE050E078
:105AC00060E070E020E030E00E941C2D1F910F91FB
:105AD0000895CF92DF92EF92FF920F931F938C0164
:105AE0009A01C62EDD24EE24FF24B701A6010E94F0
:105AF000FB2CC8010E94522D1F910F91FF90EF9037
:105B0000DF90CF9008952F923F924F925F926F92C5
:105B10007F928F929F92AF92BF92CF92DF92EF923D
:105B2000FF920F931F93DF93CF93CDB7DEB73B0167
:105B30004C0119012A016D897E898F89988D6A1916
:105B40007B098C099D09621A730A840A950AA401CB
:105B500093010E94142EE218F30804091509A80104
:105B600097010E94742E2A0D3B1D4C1D5D1DB9012D
:105B7000CA01CF91DF911F910F91FF90EF90DF90BD
:105B8000CF90BF90AF909F908F907F906F905F90DD
:105B90004F903F902F900895EF92FF920F931F9395
:105BA0007B018C01611571058105910529F420E0C7
:105BB00030E040E050E00BC00E94E201A8019701F4
:105BC0000E94742EAC01CB01DA019C01AD01B90138
:105BD000CA011F910F91FF90EF900895EF92FF92ED
:105BE0000F931F937B018C0162177307840795073E
:105BF00064F4261B370B480B590BCA01B9010E94EC
:105C0000CC2DE60EF71E081F191FB701C8011F9102
:105C10000F91FF90EF900895009729F0BC0180E06C
:105C200090E00E94E7010895629FD001739FF00108
:105C3000829FE00DF11D649FE00DF11D929FF00D1C
:105C4000839FF00D749FF00D659FF00D9927729F53
:105C5000B00DE11DF91F639FB00DE11DF91FBD01DE
:105C6000CF0111240895991B79E004C0991F96175C
:105C700008F0961B881F7A95C9F78095089597FBC1
:105C8000092E07260AD077FD04D049D006D000207F
:105C90001AF4709561957F4F0895F6F79095819568
:105CA0009F4F0895A1E21A2EAA1BBB1BFD010DC038
:105CB000AA1FBB1FEE1FFF1FA217B307E407F507BC
:105CC00020F0A21BB30BE40BF50B661F771F881F98
:105CD000991F1A9469F760957095809590959B012E
:105CE000AC01BD01CF01089597FB092E05260ED00A
:105CF00057FD04D0D7DF0AD0001C38F450954095EA
:105D0000309521953F4F4F4F5F4F0895F6F790958F
:105D10008095709561957F4F8F4F9F4F0895AA1B77
:105D2000BB1B51E107C0AA1FBB1FA617B70710F086
:105D3000A61BB70B881F991F5A95A9F780959095B8
:105D4000BC01CD010895EE0FFF1F0590F491E02DE9
:105D500009942F923F924F925F926F927F928F920F
:105D60009F92AF92BF92CF92DF92EF92FF920F93EA
:105D70001F93CF93DF93CDB7DEB7CA1BDB0B0FB6F4
:105D8000F894DEBF0FBECDBF09942A8839884888B1
:105D90005F846E847D848C849B84AA84B984C88447
:105DA000DF80EE80FD800C811B81AA81B981CE0F3E
:105DB000D11D0FB6F894DEBF0FBECDBFED01089523
:045DC000F894FFCF85
:105DC40057495A6E657400444E53206572726F725F
:105DD400203D20307800333238702D302E342E3070
:105DE40000303030303030303030303030303030DF
:105DF400303030303030303030303030303030309F
:105E0400300074632D636F6E66696730312E6B6585
:105E14006E6E656479746563686E6F6C6F67792EF6
:105E24006E65740020007003000001000000010092
:105E34000000002302BF04D3040000000012059CEC
:105E4400057D0500000100016969010000010000F1
:0E5E54000000000000000000CE2B222C3A2C93
:00000001FF
